:100000000C94ED000C940A010C940A010C940A0162
:100010000C940A010C940A010C940A010C940A0134
:100020000C940A010C940A010C940A010C940A0124
:100030000C9419070C940A010C940A010C940A01FF
:100040000C940A010C940A010C94BB190C940A013B
:100050000C940A010C940A010C940A010C940A01F4
:100060000C940A010C940A010C940A010C940A01E4
:100070000C940A010C940A010C94DA190C940A01EC
:100080000C940A010C940A010C940A011912191219
:10009000601247125A121912191260124712A5184B
:1000A00097189A18A5189F18A218A518A518AE1881
:1000B000AE18AE18AE18A81825732E2E6F25303244
:1000C00058240025732E2E6E2530325824002573B7
:1000D0002E2E4F25303258240025732E2E4E2530DB
:1000E0003258240025732E2E7A25635F2400257351
:1000F0002D4552524F52260047617465207461733A
:100100006B203D2025750D0A005543532074617303
:100110006B203D2025750D0A00496E7075742074A2
:1001200061736B203D2025750D0A0052434D2074EC
:1001300061736B203D2025750D0A0052756E206C91
:100140006564207461736B203D2025750D0A007372
:100150007461636B206F766572666C6F77202D20FB
:1001600025730D0A004D616C6C6F63206661696CCC
:1001700065640D0A002D2D2D2D2D2D2D2D2D2D2DB0
:100180002D2D205374617274696E67202573202DA4
:100190002D2D2D2D2D2D2D2D2D2D2D2D0D0A0072BA
:1001A000636D547851756575652063726561746916
:1001B0006F6E206661696C65640D0A0072636D5232
:1001C000785175657565206372656174696F6E201D
:1001D0006661696C65640D0A000011241FBECFEFD3
:1001E000D0E1DEBFCDBF12E0A0E0B1E0E6E6F1E491
:1001F00002C005900D92A032B107D9F726E0A0E227
:10020000B2E001C01D92A432B207E1F70E9473165A
:100210000C94B1200C9400000F931F93CF93DF93A5
:10022000CDB7DEB72A970FB6F894DEBF0FBECDBFAD
:1002300085E08093D70284ED92E09F938F938EEEBA
:1002400090E09F938F938E010F5F1F4F1F930F932B
:100250000E94491DC8010E946A190F900F900F90CB
:100260000F900F900F902A960FB6F894DEBF0FBE36
:10027000CDBFDF91CF911F910F9108950F931F93E1
:10028000CF93DF93CDB7DEB729970FB6F894DEBFD3
:100290000FBECDBF8091D2021F928F9384ED92E06A
:1002A0009F938F9384EE90E09F938F938E010F5FC7
:1002B0001F4F1F930F930E94491DC8010E946A1986
:1002C0000FB6F894DEBF0FBECDBF29960FB6F894D7
:1002D000DEBF0FBECDBFDF91CF911F910F9108956B
:1002E0000F931F93CF93DF93CDB7DEB729970FB648
:1002F000F894DEBF0FBECDBF8091D3021F928F93C3
:1003000084ED92E09F938F9389ED90E09F938F937C
:100310008E010F5F1F4F1F930F930E94491DC8014D
:100320000E946A190FB6F894DEBF0FBECDBF2996A2
:100330000FB6F894DEBF0FBECDBFDF91CF911F91F6
:100340000F9108950F931F93CF93DF93CDB7DEB72F
:1003500029970FB6F894DEBF0FBECDBF8BB31F92A7
:100360008F9384ED92E09F938F938EEC90E09F9318
:100370008F938E010F5F1F4F1F930F930E94491D94
:10038000C8010E946A190FB6F894DEBF0FBECDBF38
:1003900029960FB6F894DEBF0FBECDBFDF91CF9187
:1003A0001F910F9108950E9470010C94A2010F9368
:1003B0001F93CF93DF93CDB7DEB729970FB6F8948D
:1003C000DEBF0FBECDBF8F3F19F48091D90202C0AE
:1003D0008093D902282F082E000C330B3F938F9364
:1003E00084ED92E09F938F9383EC90E09F938F93A3
:1003F0008E010F5F1F4F1F930F930E94491DC8016D
:100400000E946A190FB6F894DEBF0FBECDBF2996C1
:100410000FB6F894DEBF0FBECDBFDF91CF911F9115
:100420000F9108950F931F93CF93DF93CDB7DEB74E
:1004300029970FB6F894DEBF0FBECDBF8F3F19F4DA
:100440008091D80202C08093D802282F082E000C79
:10045000330B3F938F9384ED92E09F938F9388EBC0
:1004600090E09F938F938E010F5F1F4F1F930F9309
:100470000E94491DC8010E946A190FB6F894DEBF98
:100480000FBECDBF29960FB6F894DEBF0FBECDBF0D
:10049000DF91CF911F910F910895CF93DF93EC01DE
:1004A00082E090E00E940F20888381E090E00E942B
:1004B0000F2089831A82DF91CF910895CF93DF9324
:1004C000EC01688182E090E00E942120698181E056
:1004D00090E0DF91CF910C94212083E090E00C9488
:1004E0000F20682F83E090E00C942120CF93DF93BE
:1004F000EC0148E050E060E370E00E94FF1F1886C6
:10050000DF91CF91089548E050E060E370E00C94F3
:1005100017200F931F93CF93DF938C01EB0189E09A
:10052000E1EAF1E0DB0101900D928A95E1F7C80163
:100530000E940F208F3F71F08983B8016F5F7F4F5A
:1005400043E050E0CE010496DF91CF911F910F91CF
:100550000C94FF1F89E0FE0111928A95E9F7DF9163
:10056000CF911F910F9108950E940F209FEF980F38
:1005700081E09E3F08F080E008950F931F93CF9392
:10058000DF9303EB14E0C4E0D1E0B801CE010E9498
:100590008902B8016E5E7F4FCE0108960E948902E3
:1005A000B801675F7F4FCE0180589F4F0E9489023C
:1005B000B801655E7F4FCE0188579F4F0E94890228
:1005C00060960C5D1F4FC43881E0D807F1F6DF91CB
:1005D000CF911F910F9108950F931F93CF93DF93A6
:1005E00009E113E0C0E0D1E0B801CE010E94890228
:1005F000B8016E5E7F4FCE0108960E948902B80155
:10060000675F7F4FCE0180589F4F0E948902B801DB
:10061000655E7F4FCE0188579F4F0E94890260968A
:100620000C5D1F4FC03881E0D807F1F6DF91CF9104
:100630001F910F910895EF92FF921F93CF93DF9335
:1006400053E9E52E54E0F52EC0EDD0E0CE010E9436
:100650000F20182FCE0140970E940F20212F30E04D
:10066000322F2227282BF70131832083CE01809659
:100670000E940F20182FCE0140960E940F20212F9C
:1006800030E0322F2227282BF70133832283219653
:10069000F4E0EF0EF11CC83DD105C1F6DF91CF911A
:1006A0001F91FF90EF900895AF92BF92CF92DF928B
:1006B000FF920F931F93CF93DF93C9E3D4E000E43D
:1006C00010E089E0F82E89E0EBEAF1E0DE0101902C
:1006D0000D928A95E1F7C8010E940F208F3F41F0EB
:1006E00043E050E0B801CE0104960E94FF1F05C010
:1006F000FE018F2D11928A95E9F76E01E9E0CE0E89
:10070000D11C89E0EBEAF1E0D60101900D928A95C7
:10071000E1F75801F0E2AF0EB11CC5010E940F20B5
:100720008F3F41F043E050E0B501CE010D960E94AD
:10073000FF1F05C0F6018F2D11928A95E9F7629689
:100740000D5F1F4F0F34110509F0BDCFDF91CF9121
:100750001F910F91FF90DF90CF90BF90AF900895C1
:100760006AED72E08CE890E00E94890263EE72E02C
:100770008CE990E00E9489026CEE72E08CEA90E0D5
:100780000E94890265EF72E08CEB90E00E94890282
:100790006EEF72E08CEC90E00E94890267E073E0FB
:1007A0008CED90E00E94890260E173E08CEE90E0B5
:1007B0000C948902CF93DF9385E090E00E940F2094
:1007C000C3EDD5E0888386E090E00E940F20898306
:1007D00087E090E00E940F208A8388E090E00E94EA
:1007E0000F208B8389E090E00E940F208C838AE0A9
:1007F00090E00E94B4028D838BE090E00E940F2075
:100800008E838CE090E00E94B4028F8386E190E0BA
:100810000E940F20888787E190E00E940F2089873F
:1008200088E190E00E940F208A8789E190E00E9491
:100830000F208B878AE190E00E940F208C87DF9148
:10084000CF9108950C940F200C942120CF93DF9327
:10085000CDB7DEB72C970FB6F894DEBF0FBECDBF75
:10086000CE010A960E944D028A858F3F19F08B8532
:100870008F3F21F485EB91E00E945E020E946D02A1
:100880008F3F19F485E50E947102CE0101960E9406
:10089000760248E050E068EB71E0CE0101960E94DC
:1008A000D61C892B21F088EB91E00E9483020E94E4
:1008B000BD020E94EC020E946D02853511F40E9477
:1008C0001B030E946D02873431F40E9454030E947E
:1008D000B0030E94DA032C960FB6F894DEBF0FBE69
:1008E000CDBFDF91CF910895CF93DF938CE090E05F
:1008F0000E941C07EC01009731F0FC01119211924B
:10090000CF010E945405CE01DF91CF910895AF929F
:10091000BF92CF92DF92EF92FF920F931F93CF93EC
:10092000DF936C017B01B42EA22E0E941B0CF601FA
:10093000C081D181CE018E219F21A11003C0892BBE
:1009400021F43BC0E816F906C1F5BB2041F0C70110
:10095000809590958C239D23F6019183808300E000
:1009600010E00E942C0D012B09F43DC0811102C042
:100970000E9464060E94A91091FD1CC00FB6F89455
:100980000F92F60180819181970128233923A110CC
:1009900003C0232B21F40CC0E216F30649F4BB205C
:1009A00039F0E094F094E822F922F601F182E08235
:1009B0000F900FBEEC01DD2716C00115110589F25D
:1009C000BB2019F060E071E002C060E070E0A110AF
:1009D00074606E297F29A801C60102960E947D0ECF
:1009E000C0E0D0E0BECFCE01DF91CF911F910F913B
:1009F000FF90EF90DF90CF90BF90AF900895CF928F
:100A0000DF92EF92FF920F931F93CF93DF938C01AE
:100A1000EB017C0185E0E80EF11C0E941B0CD80163
:100A20001796ED91FC9118978D919C911197C82B79
:100A3000D92BCD93DC93C0E0D0E0D8016D917C91AF
:100A40001197EE15FF05E1F0D280C380208131813E
:100A5000C9019927AC014623572332FD03C0452B1A
:100A600021F40BC08417950741F430FF02C0C82B56
:100A7000D92B7260CF010E94B60FED2DFC2DDDCF7A
:100A8000C095D0956C237D236D937C930E942C0D93
:100A9000F80180819181DF91CF911F910F91FF909B
:100AA000EF90DF90CF900895FC01039692838183AD
:100AB0002FEF3FEF3483238396838583908787834B
:100AC00010820895FC011186108608950F931F93DC
:100AD000CF93DF938C01FB01808191818F3F2FEFBA
:100AE000920721F4E801AF81B8850EC0D8011396B2
:100AF00012962D913C911397E901488159818417F1
:100B0000950710F0D901F4CF12968D919C9113970F
:100B100093838283EC01FD83EC83B583A4831396D6
:100B2000FC93EE93129711870087F80180818F5F05
:100B30008083DF91CF911F910F910895CF93DF9321
:100B4000FC01A085B1858281938124813581EC01EE
:100B50003D832C83C481D5819B838A8311968D919B
:100B60009C911297E817F90721F41296DC93CE9323
:100B70001197118610868C9181508C938C91DF9106
:100B8000CF91089531E1FC013083319722E2208337
:100B90003197A3E3A08331976083319770833197B6
:100BA0001082319760E8608331971082319762E05C
:100BB0006083319763E06083319764E060833197AD
:100BC00065E06083319766E06083319767E060831A
:100BD000319768E06083319769E06083319760E125
:100BE000608331973083319732E13083319733E13D
:100BF0003083319734E13083319735E13083319759
:100C000036E13083319737E13083319738E13083F3
:100C1000319739E13083319730E23083319731E2D7
:100C2000308331972083319723E2208331974083AB
:100C300031975083319726E22083319727E2208332
:100C4000319728E22083319729E22083319720E3EE
:100C50002083319721E320838697089583E08BBD1D
:100C600087EE8ABD8BE08EBD87B7806187BFA0917C
:100C70008E02B0918F02CD91CDBFDD91DEBFFF918D
:100C8000EF91DF91CF91BF91AF919F918F917F9124
:100C90006F915F914F913F912F911F910F91FF9015
:100CA000EF90DF90CF90BF90AF909F908F907F900C
:100CB0006F905F904F903F902F901F900F900FBEBE
:100CC0000F90089581E008950F920FB6F8940F9257
:100CD0001F9211242F923F924F925F926F927F92B8
:100CE0008F929F92AF92BF92CF92DF92EF92FF923C
:100CF0000F931F932F933F934F935F936F937F9324
:100D00008F939F93AF93BF93CF93DF93EF93FF9313
:100D1000A0918E02B0918F020DB60D920EB60D927B
:100D20000E940E0EA0918E02B0918F02CD91CDBF88
:100D3000DD91DEBFFF91EF91DF91CF91BF91AF9138
:100D40009F918F917F916F915F914F913F912F91E3
:100D50001F910F91FF90EF90DF90CF90BF90AF90D9
:100D60009F908F907F906F905F904F903F902F90CB
:100D70001F900F900FBE0F9008950F920FB6F8942A
:100D80000F921F9211242F923F924F925F926F9277
:100D90007F928F929F92AF92BF92CF92DF92EF920B
:100DA000FF920F931F932F933F934F935F936F93F4
:100DB0007F938F939F93AF93BF93CF93DF93EF93E3
:100DC000FF93A0918E02B0918F020DB60D920EB6D8
:100DD0000D920E942B0C81110E940E0EA0918E028A
:100DE000B0918F02CD91CDBFDD91DEBFFF91EF912C
:100DF000DF91CF91BF91AF919F918F917F916F9133
:100E00005F914F913F912F911F910F91FF90EF9024
:100E1000DF90CF90BF90AF909F908F907F906F901A
:100E20005F904F903F902F901F900F900FBE0F90AC
:100E300008950E94BD061895CF93DF93EC010E94A0
:100E40001B0CCE010E94B71AEC010E942C0D2097BA
:100E500011F40E941117CE01DF91CF910895CF9325
:100E6000DF93009751F0EC010E941B0CCE010E9411
:100E70004F1BDF91CF910C942C0DDF91CF910895F2
:100E80000FB6F8940F92FC01928D0F900FBE81E087
:100E9000911180E008950F931F93CF93DF93EC019E
:100EA000042F1A8D4C8D4423B1F150E0011115C06F
:100EB0008A819B810E94E31C2C8D8A819B81820FF9
:100EC000911D9B838A832C813D818217930718F1A2
:100ED000888199819B838A831EC08E819F810E9415
:100EE000E31C8C8D90E09195819591092E813F8135
:100EF000280F391F3F832E834881598124173507D6
:100F000030F42C813D81820F931F9F838E830230AA
:100F100011F4111111501F5F1A8F80E0DF91CF91F2
:100F20001F910F910895FC01CB01448D4423A1F042
:100F300050E026813781240F351F37832683648153
:100F400075812617370720F020813181378326836A
:100F5000668177810C94E31C0895EF92FF921F93B2
:100F6000CF93DF93EC010FB6F8940F921E8D7C01A6
:100F700081E1E80EF11C11165CF48989882341F0A7
:100F8000C7010E940A0F81110E9481101150F3CFF6
:100F90008FEF8E8F0F900FBE0FB6F8940F921D8DAE
:100FA0007E0188E0E80EF11C11165CF48885882328
:100FB00041F0C7010E940A0F81110E948110115057
:100FC000F3CF8FEF8D8F0F900FBEDF91CF911F91D9
:100FD000FF90EF900895CF93DF93EC01892B09F4F4
:100FE0003EC09B8D992309F43AC07C8D0FB6F894CE
:100FF0000F92488159819A01979F200D311D11242C
:101000003D832C831A8E5B834A83892F90E001975E
:10101000789F9001799F300D1124CA01820F931F90
:101020009F838E838FEF8D8F8E8F61110CC088858B
:10103000882389F0CE0108960E940A0F882359F070
:101040000E94640608C0CE0108960E945405CE0195
:1010500041960E9454050F900FBE81E001C080E0D0
:10106000DF91CF910895FF920F931F93CF93DF935A
:10107000811103C0C0E0D0E01BC0F42E162F082F52
:10108000869FC001112481960E941C07EC010097E5
:1010900089F3111103C09983888303C081969983D2
:1010A00088830B8F1C8F61E0CE010E94EB07F8A2B2
:1010B000CE01DF91CF911F910F91FF900895AF92D4
:1010C000BF92CF92DF92FF920F931F93CF93DF9344
:1010D00000D000D01F92CDB7DEB78C016B015D83CD
:1010E0004C83F22E80E0580198E0A90EB11C0FB697
:1010F000F8940F92F801228D938D291718F0F2E0E1
:10110000FF1214C04F2DB601C8010E944B07F80111
:101110009189992321F0C80141960E940A0F8111FB
:101120000E9464060F900FBE81E050C02C813D816B
:10113000232B19F40F900FBE48C0811104C0CE01BB
:1011400001960E9444100F900FBE0E941B0C0FB618
:10115000F8940F92F801858D8F3F09F4158EF801F0
:10116000868D8F3F09F4168E0F900FBEBE016C5F07
:101170007F4FCE0101960E944F10811121C00FB602
:10118000F8940F92F801928D0F900FBE838D9813F3
:1011900011C06C817D81C5010E946C0EC8010E9446
:1011A000AD070E942C0D882311F081E0A0CF0E9492
:1011B0006406FBCFC8010E94AD070E942C0DF5CF3D
:1011C000C8010E94AD070E942C0D80E00F900F9087
:1011D0000F900F900F90DF91CF911F910F91FF9083
:1011E000DF90CF90BF90AF900895EF92FF921F9342
:1011F000CF93DF93EC019A8D8B8D981710F02230EE
:10120000E9F47A011E8D8A8D422FCE010E944B0790
:101210001F3F81F48989882379F0CE0141960E948D
:101220000A0F882349F0E114F10431F081E0F7015D
:10123000808305C01F5F1E8F81E001C080E0DF91C9
:10124000CF911F91FF90EF900895AF92BF92CF92F0
:10125000DF92FF920F931F93CF93DF9300D000D0C4
:101260001F92CDB7DEB78C016B015D834C8380E0AC
:10127000580191E1A90EB11C0FB6F8940F92F80134
:10128000F28CFF20A9F0B601C8010E949307FA94DE
:10129000F801F28E8085882339F0C80108960E94F3
:1012A0000A0F81110E9464060F900FBE81E050C0AA
:1012B0002C813D81232B19F40F900FBE48C0811162
:1012C00004C0CE0101960E9444100F900FBE0E94F0
:1012D0001B0C0FB6F8940F92F801858D8F3F09F41F
:1012E000158EF801868D8F3F09F4168E0F900FBE74
:1012F000BE016C5F7F4FCE0101960E944F1081119D
:101300001CC0C8010E944007882389F06C817D8140
:10131000C5010E946C0EC8010E94AD070E942C0DF1
:10132000882311F081E0A8CF0E946406FBCFC8019A
:101330000E94AD070E942C0DF5CFC8010E94AD0799
:101340000E942C0DC8010E944007882359F380E0B9
:101350000F900F900F900F900F90DF91CF911F91F2
:101360000F91FF90DF90CF90BF90AF9008956115DF
:10137000710549F1A0EEB5E020E030E0E0E0F0E0FA
:1013800012964D915C9113974817590741F4F90152
:10139000EE0FFF1FEE0FFF1FE052FA4F10C0309705
:1013A00031F44D915C911197452B09F4FD012F5FAC
:1013B0003F4F14962A30310519F7309721F0718389
:1013C0006083938382830895CF93DF93EC010FB6FC
:1013D000F8940F928D8D8F3F09F41D8E8E8D8F3F67
:1013E00009F41E8E0F900FBE8A8D811104C0CE01AC
:1013F00041960E94C20ECE01DF91CF910C94AD07B1
:10140000E0914D02F0914E028081811103C08FEF77
:101410009FEF09C0E0914D02F0914E020580F681E8
:10142000E02D80819181909324028093230208957E
:10143000FF920F931F93CF93DF93EC01F62E009151
:101440002C0210912D0280918E0290918F020296B3
:101450000E949E05CF3F8FEFD807C1F5FF20B1F165
:10146000E0913002F0913102A0918E02B0918F0292
:101470001596FC93EE931497A0918E02B0918F0273
:101480008481958117969C938E93169780918E02F6
:1014900090918F02A481B581029613969C938E93AE
:1014A000129780918E0290918F0202969583848389
:1014B000E0918E02F0918F028FE292E09387828713
:1014C00080912F028F5F80932F022FC0C00FD11FFA
:1014D000E0918E02F0918F02D383C28360918E02DD
:1014E00070918F02C017D10768F480914B029091E0
:1014F0004C026E5F7F4FDF91CF911F910F91FF9054
:101500000C94660580914D0290914E026E5F7F4F64
:101510000E9466058091230290912402C817D90782
:1015200020F4D0932402C0932302DF91CF911F9126
:101530000F91FF90089580913802882309F10FB62A
:10154000F8940F92E0913E02F0913F02C681D7815C
:10155000CE0102960E949E0580912E0281508093BA
:101560002E02809138028150809338020F900FBE76
:101570008F89988D0E942F07CE010E942F07DBCF05
:1015800080916102823010F00E9464060E947B17F5
:10159000D2CF5F926F927F928F929F92AF92BF92C3
:1015A000CF92DF92EF92FF920F931F93CF93DF932F
:1015B0003C016B015A014901502ECA010E941C07CF
:1015C0008C01892B09F4F9C088E290E00E941C0785
:1015D000EC01892BC9F0188F0F8BA50165EA70E02B
:1015E000C8010E94EC1C81E0A81AB1088F89988D6F
:1015F000A80EB91EC114D104C9F0BE01675E7F4FA9
:10160000F601C601089607C0C8010E942F07D5C081
:101610008E179F0749F09F014191DB014D93BD015A
:10162000D9012C912111F4CF18A201C0198E052DDA
:10163000053008F004E00E8B6E01B2E0CB0ED11C39
:10164000C6010E946205CE010C960E946205D987F0
:10165000C88785E090E0801B91099D878C87DB8B94
:10166000CA8B84E0FE01B396DF011D928A95E9F7EB
:101670001FA2A401B301C5010E94C20599838883FA
:10168000E114F10419F0F701D183C0830FB6F89487
:101690000F9280912E028F5F80932E0280918E0296
:1016A00090918F02892BC1F5D0938F02C0938E0247
:1016B00080912E02813009F03FC001E612E08EE8F1
:1016C000E82E82E0F82EC8010E945405075F1F4FE4
:1016D000E016F106C1F788E592E00E9454058FE418
:1016E00092E00E94540582E492E00E94540589E34E
:1016F00092E00E9454058FE292E00E94540588E532
:1017000092E090934E0280934D028FE492E090938A
:101710004C0280934B0210C080912A0281110CC0B0
:10172000E0918E02F0918F0296898E89891720F0C0
:10173000D0938F02C0938E02809125028F5F809399
:10174000250289A3EE8980912B028E1710F4E09375
:101750002B0289E08E9FF0011124EF59FD4F01808B
:10176000F281E02DFD83EC83248135813F832E833C
:10177000A481B5811396DC92CE921297D582C48251
:10178000EE898E9FF0011124EF59FD4FFB87EA8708
:1017900080818F5F80830F900FBE80912A02882303
:1017A00051F0E0918E02F0918F0296898E89981700
:1017B00010F40E94640681E001C08FEFDF91CF91A9
:1017C0001F910F91FF90EF90DF90CF90BF90AF905F
:1017D0009F908F907F906F905F900895EF92FF920F
:1017E0000F9381E2E82E82E0F82E00E020E030E066
:1017F00040E450E061EC71E08BE99AE00E94C90A94
:10180000813099F40E946412813079F4F8942FEFBA
:101810003FEF309324022093230280932A021092F8
:101820002D0210922C020E942E06809106010F912B
:10183000FF90EF900895809120028F5F80932002A7
:1018400008950FB6F8940F9280912C0290912D027A
:101850000F900FBE0895CF92DF92EF92FF920F93F9
:101860001F93CF93DF93809120028111E2C0C0913A
:101870002C02D0912D026E018FEFC81AD80AD09297
:101880002D02C0922C02C114D104B9F480914D02F2
:1018900090914E0220914B0230914C0230934E02B7
:1018A00020934D0290934C0280934B02809126022C
:1018B0008F5F809326020E94000A809123029091FC
:1018C0002402C816D90608F49EC080E069E0E091C1
:1018D0004D02F0914E029081911103C02FEF3FEF26
:1018E0000FC0E0914D02F0914E020580F681E02D8F
:1018F0000680F781E02D22813381C216D30628F4B9
:1019000030932402209323027FC0C285D385248193
:10191000358146815781D90115965C934E93149772
:1019200046815781DA0113963C932E9312979F01BB
:101930002E5F3F4F09811A810217130711F45A8352
:10194000498313861286988191509883A489B5891A
:101950001097F9F04685578500891189EA011D83A2
:101960000C8300891189E8015B834A831196ED900D
:10197000FC901297AF01445F5F4FE416F50621F427
:1019800012961C930E931197158A148A9C9191506C
:101990009C93A68990912B029A1710F4A0932B0286
:1019A0006A9FD0011124AF59BD4F11960D90BC9183
:1019B000A02DB583A48314964D915C911597578300
:1019C000468314964D915C911597EA013B832A83D7
:1019D00015963C932E931497A6896A9FD0011124E3
:1019E000AF59BD4FB387A2879C919F5F9C93A091F5
:1019F0008E02B0918F02268956969C91291708F481
:101A000066CF81E064CF80E0E0918E02F0918F029A
:101A1000E689D9E0ED9FF0011124EF59FD4F908147
:101A2000923008F081E090912702992361F081E0E3
:101A30000AC0809128029091290201969093290270
:101A40008093280280E0DF91CF911F910F91FF904A
:101A5000EF90DF90CF900895EF92FF920F931F9336
:101A6000CF93DF930FB6F8940F92809120028150AC
:101A70008093200280912002882311F080E0B0C082
:101A800080912E028823D1F3E0904702F090480223
:101A9000E0E0F0E039E041E080914202882309F47F
:101AA00081C0D7011696ED91FC911797A489B5894D
:101AB0006685778580899189EB019D838C838089F8
:101AC0009189EC017B836A83BF01645F7F4F11962C
:101AD0000D911C9112970617170721F412969C93EB
:101AE0008E931197158A148A8C9181508C93A285BC
:101AF000B3858481958166817781EC017D836C83D8
:101B000066817781EB019B838A83CF0102961196D0
:101B10000D911C9112970817190721F412967C93C6
:101B20006E931197138612862C9121502C93A689BF
:101B300020912B022A1710F4A0932B023A9FD00178
:101B40001124AF59BD4F11960D90BC91A02DB583B6
:101B5000A48314966D917C91159777836683149670
:101B60006D917C911597EB019B838A8315969C93CD
:101B70008E931497A6893A9FD0011124AF59BD4F77
:101B8000B387A2878C918F5F8C93A0918E02B091C6
:101B90008F02968956968C91981708F47DCF4093C2
:101BA00027027ACFEF2B11F00E94000AC091280281
:101BB000D0912902209761F011E00E942B0C811135
:101BC000109327022197C9F7109229021092280238
:101BD00080912702882309F451CF0E94640681E096
:101BE0000F900FBEDF91CF911F910F91FF90EF905B
:101BF0000895CF93DF93EC01892B19F40E946406BA
:101C00000AC00E941B0C60E0CE010E94180A0E94CC
:101C10002C0D882399F3DF91CF91089580912002B4
:101C2000882321F081E080932702089510922702F3
:101C3000A0918E02B0918F02E0918E02F0918F02FE
:101C40002D913C918789908D8217930760F0609168
:101C50008E0270918F0280918E0290918F02675E4A
:101C60007F4F0E941B1780912B0269E0482F50E0A4
:101C7000649F9001659F300D1124F901EF59FD4FCC
:101C80009081911102C08150F1CFA181B281129651
:101C90000D90BC91A02DB283A1832C593D4FA2176A
:101CA000B30731F412962D913C911397328321831F
:101CB00099E0949FF001959FF00D1124EF59FD4F8D
:101CC0000180F281E02D2681378130938F022093AD
:101CD0008E0280932B020895CF93DF93EB016091E6
:101CE0008E0270918F02645F7F4F0E94660561E0F3
:101CF000CE01DF91CF910C94180ACF93DF93FC01B2
:101D0000A0918E02B0918F0270681D967C936E93A5
:101D10001C97A181B281C0918E02D0918F02BF87A2
:101D2000AE87C0918E02D0918F0214968D919C91B6
:101D30001597998B888B20918E0230918F02149683
:101D4000CD91DC911597245F3F4F3B832A832091EF
:101D50008E0230918F02245F3F4F15963C932E9355
:101D60001497A0918E02B0918F025596FC93EE933A
:101D7000549790819F5F908361E0CA01DF91CF917A
:101D80000C94180A0F931F93CF93DF93FC018B01E0
:101D9000A181B28180918E0290918F02EC01BF8768
:101DA000AE8780918E0290918F0214962D913C9176
:101DB0001597EC01398B288B20918E0230918F0280
:101DC00014968D919C911597245F3F4FEC013B83B6
:101DD0002A8320918E0230918F02245F3F4F159607
:101DE0003C932E931497A0918E02B0918F0255963A
:101DF000FC93EE93549790819F5F9083442311F05E
:101E00000FEF1FEF642FC801DF91CF911F910F914A
:101E10000C94180ACF93DF93DC011596ED91FC9199
:101E200016970680F781E02DA489B5898685978568
:101E300020893189EC013D832C83C089D1899B8322
:101E40008A83CF010C9611962D913C9112972817F9
:101E5000390721F41296DC93CE931197158A148AD0
:101E60002C9121502C932091200221114FC0A2854A
:101E7000B3858481958126813781EC013D832C8354
:101E8000C681D7819B838A839F012E5F3F4F119626
:101E90008D919C9112978217930721F41296DC93EF
:101EA000CE931197138612868C9181508C93A689BC
:101EB00080912B028A1710F4A0932B0289E08A9F4D
:101EC000D0011124AF59BD4F11960D90BC91A02D9A
:101ED000B583A48314964D915C91159757834683DF
:101EE0001496CD91DC9115973B832A8315963C93EC
:101EF0002E931497A6898A9FD0011124AF59BD4F04
:101F0000B387A2878C918F5F8C931FC0A0914302EF
:101F1000B0914402B787A68714962D913C911597EE
:101F2000318B208B1496CD91DC9115979B838A83FE
:101F300015969C938E93149782E492E0958B848BF4
:101F4000809142028F5F80934202A0918E02B091F5
:101F50008F02968956968C91891720F481E08093A0
:101F6000270201C080E0DF91CF910895CF93DF93E6
:101F7000DC01706811967C936E931696ED91FC913E
:101F8000179718964D915C91199712962D913C9147
:101F9000139714968D919C911597E9019D838C83DD
:101FA00014968D919C911597EC013B832A83EA014D
:101FB00029813A81A217B30711F49A83898319966C
:101FC0001C921E921897DA018C9181508C93A285F5
:101FD000B3858481958126813781EC013D832C83F3
:101FE000C681D7819B838A839F012E5F3F4F1196C5
:101FF0008D919C9112978217930721F41296DC938E
:10200000CE931197138612868C9181508C93A6895A
:1020100080912B028A1710F4A0932B0289E08A9FEB
:10202000D0011124AF59BD4F11960D90BC91A02D38
:10203000B583A48314964D915C911597578346837D
:102040001496CD91DC9115973B832A8315963C938A
:102050002E931497A6898A9FD0011124AF59BD4FA2
:10206000B387A2878C918F5F8C93A0918E02B091E1
:102070008F02968956968C91891718F481E0809387
:102080002702DF91CF91089520912602FC01208341
:1020900020912C0230912D02328321830895CF9319
:1020A000DF930FB6F8940F9240912C0250912D02BD
:1020B000DB012D913C912F3FBFEF3B07E1F0EC019D
:1020C000E981FA81A0912602B881BA1741F04E1732
:1020D0005F0728F0FB011182108281E00DC04E1BCA
:1020E0005F0B42175307B0F7FB01241B350B3183FD
:1020F00020830E94441080E00F900FBEDF91CF91AB
:10210000089581E0809327020895009721F480913B
:102110008E0290918F02DC015796ED91FC915897B9
:1021200080E090E0DC012191253A21F40196A11D87
:10213000B11DF9CF089580912A02882331F0809152
:102140002002882321F080E0089581E0089582E054
:102150000895E0918E02F0918F0284859585E0913B
:102160008E02F0918F02A0918E02B0918F0256964E
:102170004C9125E030E0241B3109358724870895F0
:102180000FB6F8940F928091940290919502892B4A
:1021900019F583EA92E00E9454058AE992E00E94D0
:1021A000540583EA92E090939902809398028AE919
:1021B00092E0909397028093960240E065E085E07C
:1021C0000E9433089093950280939402009721F027
:1021D00065ED71E00E94B7090F900FBE0895FC01F4
:1021E00073836283918780874617570778F0421B75
:1021F000530B8485958548175907C8F4BF016E5F56
:102200007F4F80919602909197020DC0421753071D
:1022100018F46217730758F4BF016E5F7F4F809107
:102220009802909199020E94660580E0089581E0ED
:102230000895EF92FF920F931F93CF93DF93EC01DA
:102240008B017A016C857D85600F711F9801A70154
:10225000CE010E94EF10882349F08C859D85080FE0
:10226000191FE889F989CE010995ECCFDF91CF914B
:102270001F910F91FF90EF900895EF92FF920F93AF
:102280001F93CF93DF938C017B01E0919802F09133
:1022900099020580F681E02DC681D781CE01029694
:1022A0000E949E058B8982FF06C0A701B801CE015E
:1022B0000E94191102C08E7F8B8BE889F989CE01AB
:1022C000DF91CF911F910F91FF90EF900994E091D2
:1022D0009802F09199028081882351F00580F6815F
:1022E000E02D6FEF7FEF808191810E943D11EFCF54
:1022F0008091960290919702909399028093980210
:10230000F0939702E09396020895CF93DF9300D065
:1023100000D01F92CDB7DEB7E0919802F0919902FC
:10232000D080DD2031F00580F681E02D0081118123
:1023300002C000E010E00E941B0C0E94210C7C01F6
:102340008091900290919102E816F90620F40E9483
:10235000671181E001C080E0F0929102E09290026A
:10236000811124C0DD2051F0E016F10670F00E94CA
:102370002C0DB701C8010E943D111EC0E0919602CC
:10238000F0919702808141E0811140E0B8016E191F
:102390007F0980919402909195020E94E4090E9425
:1023A0002C0D811109C00E94640606C00E942C0DEC
:1023B00003C0898187FF0EC040E050E0BE016F5F1F
:1023C0007F4F80919402909195020E94250981117E
:1023D000F0CFA2CF0C811D81D8011A968D919C91CE
:1023E0001B97892B21F0C80102960E949E050E942E
:1023F000210C7C018091900290919102E816F906DF
:1024000010F40E946711F0929102E0929002E9812B
:102410008E2FEE0F990BAA0BBB0BFC013197E93005
:10242000F10550F6EA5BFF4FD80153968C910C945E
:10243000B11A8160F801838B2A813B81648575859F
:10244000620F731FA701C8010E94EF10882309F4CF
:10245000B3CFD80153968C91539782FF0DC06A81F8
:102460007B811C968D919C911D97680F791FA70108
:10247000C8010E94191103C08E7FF801838BD80117
:102480005096ED91FC915197C801099595CF8160C7
:10249000D80153968C9353976A817B811D967C93C8
:1024A0006E931C976E0D7F1D9701A701C8010E94B6
:1024B000EF1082CF81FD04C0C8010E942F077CCF9E
:1024C0008E7FF801838B78CFEF92FF920F930E945B
:1024D000C0108091940290919502892B81F082E93D
:1024E000E82E82E0F82E02E020E030E040E850E004
:1024F0006AED71E085E891E10E94C90A01C080E0BF
:102500000F91FF90EF9008958F929F92AF92BF929C
:10251000CF92DF92FF920F931F93CF93DF934C01E3
:102520005B01F42E690184E190E00E941C07EC013C
:10253000892BA1F01B8A0E94C01099828882BD86D7
:10254000AC86DF86CE86198B088BCE0102960E9460
:102550006205FF2019F08B8984608B8BCE01DF919F
:10256000CF911F910F91FF90DF90CF90BF90AF90D0
:102570009F908F9008950F931F93CF93DF9300D078
:1025800000D01F92CDB7DEB7A0919402B091950212
:10259000109729F1F90169835B834A839D838C83BA
:1025A0006630A4F40E949B10E0919402F091950291
:1025B00020E0823011F4A80102C040E050E0BE01EA
:1025C0006F5F7F4FCF010E945F080AC020E0AF011C
:1025D000BE016F5F7F4FCD010E94F50801C080E012
:1025E0000F900F900F900F900F90DF91CF911F9150
:1025F0000F9108950FB6F8940F920F900FBEFC0143
:102600008685978508950FB6F8940F92FC01778719
:1026100066870F900FBE0895E7E0F1E020E030E01C
:10262000908198130CC09181961309C047E0429F96
:10263000C001439F900D1124895F9E4F08952F5F25
:102640003F4F37962431310559F780E090E00895E7
:102650000F931F9300E010E020E030E040E050E0F6
:1026600063E080910C0690910D060E94BB121F91B1
:102670000F9108950C9428130E942813DA98089556
:102680000F931F93CF93DF93EC010E942813BE0199
:1026900080910C0690910D060E9403130E94210C5C
:1026A00000E010E020E030E0AC0161E080910C0639
:1026B00090910D060E94BB12DF91CF911F910F9157
:1026C0000895CF93C82FDA9AD89A8091DC052AE032
:1026D000829FC001112496958795969587950E94B3
:1026E000F90DD8988C2F90E0CF910C944013CF9394
:1026F000C82FE0910A06F0910B068081853021F405
:102700008091DA058111DA9865E081E00E940C136E
:1027100090930B0680930A068C2F90E0CF910C9437
:102720004013CF93C82FDA9A9091D8058091DC0599
:10273000992369F0D9982AE0829FC00111249695C7
:102740008795969587950E94F90DD99A0CC0D99ACC
:102750002AE0829FC00111249695879596958795CA
:102760000E94F90DD9988C2F90E0CF910C944013D2
:1027700020E1829FC001112499276F709C01262BB4
:10278000B90180910806909109060C94FF04CF933B
:10279000C82F0E94D701E0910A06F0910B068081B4
:1027A0006C2F0E940C1390930B0680930A06FC0179
:1027B0002281222329F080816C2FCF910C94B813B1
:1027C000CF9108950F931F9398B382E0892788BB18
:1027D00080910C0690910D060E94FA12BC01615086
:1027E000710980910C0690910D0661157105A1F497
:1027F00000E010E020E030E040E050E063E00E94C4
:10280000BB12C19AE0910A06F0910B0661818081AA
:102810001F910F910C94B8131F910F910C940313F7
:102820000F931F930E9474049093090680930806E7
:1028300002EE13E120E030E041E06AEF70E082EE6A
:1028400091E00E94841290930D0680930C061F91D4
:102850000F910895DA9A8091D8058111D99A65E08F
:1028600081E00E940C1390930B0680930A060FEFF1
:102870001FEF20E041E06FEF70E08091080690913B
:1028800009060E948704682F6F7024E0969587954B
:102890002A95E1F78F700E940C13DC0190930B06D0
:1028A00080930A06892B19F313968D919C911497A6
:1028B000892B51F01396ED91FC91149715960D907C
:1028C000BC91A02D8C910995E0910A06F0910B0620
:1028D00080810E941202CBCF883091056CF45BB3EB
:1028E00021E030E0B90102C0660F771F8A95E2F758
:1028F000CB01852B8BBB08950C940C01883091057E
:1029000074F44BB321E030E0B90102C0660F771FC9
:102910008A95E2F7CB01809584238BBB08950C94B4
:102920000C01883091056CF45BB321E030E0B90113
:1029300002C0660F771F8A95E2F7CB0185278BBB14
:1029400008950C940C01C09AC19AC29AC39AC49A71
:10295000C59AC69AC79A08955F926F927F928F9296
:102960009F92AF92BF92CF92DF92EF92FF920F931E
:102970001F93CF93DF9353B28091D302581609F47B
:1029800065C1C9E1D3E0A3E0AA2EA4E0BA2EB3E961
:10299000EB2EB4E0FB2E00E010E0652C712C809152
:1029A000D30290E0002E02C0959587950A94E2F735
:1029B00080FD8DC0C301002E02C0959587950A94B5
:1029C000E2F780FF08C18881882319F0CE010E94B8
:1029D0006A198985882321F0CE0109960E946A1917
:1029E0008091D202853509F05BC0CC24C394D12CF0
:1029F000460181E0881A9108F701808191819C014C
:102A0000082C02C0369527950A94E2F720FF0DC0E6
:102A10000C2C02C0969587950A94E2F780FD05C0BC
:102A2000C401959587950E946C14F701808191816E
:102A30009C01082C02C0369527950A94E2F720FDE8
:102A40000DC00C2C02C0969587950A94E2F780FF82
:102A500005C0C401959587950E947E14F701808179
:102A600091819C01082C02C0369527950A94E2F7C3
:102A70000C2C02C0969587950A94E2F7822B932B33
:102A800080FD05C0C401959587950E949114F2E0E0
:102A9000CF0ED11C81E1C816D10409F0A9CF0CC01A
:102AA000873451F4033011053CF0F501808188230F
:102AB00019F0C5010E9477198091D30290E0002E91
:102AC00002C0959587950A94E2F780FF84C0C30100
:102AD000002E02C0959587950A94E2F780FD7BC091
:102AE0008A89882321F0CE0142960E946A198B8D33
:102AF000882321F0CE014B960E946A198091D20260
:102B0000853509F05BC0CC24C394D12C4601F1E09B
:102B10008F1A9108F701828193819C01082C02C0D1
:102B2000369527950A94E2F720FF0DC00C2C02C0C1
:102B3000969587950A94E2F780FD05C0C4019595A6
:102B400087950E946C14F701828193819C01082C67
:102B500002C0369527950A94E2F720FD0DC00C2C93
:102B600002C0969587950A94E2F780FF05C0C401DC
:102B7000959587950E947E14F701828193819C012F
:102B8000082C02C0369527950A94E2F70C2C02C057
:102B9000969587950A94E2F7822B932B80FD05C0CA
:102BA000C401959587950E949114F2E0CF0ED11C37
:102BB00081E1C816D10409F0A9CF0DC0873459F4BA
:102BC0000330110544F0F5018185882321F0C5010A
:102BD00009960E9477190F5F1F4FA496F2E1AF0E7E
:102BE000B11C84E0E80EF11C0830110509F0D7CEC5
:102BF0008091D2028734B9F4852D87709091DD05DC
:102C0000891302C082E00DC09091DE05891302C0D5
:102C100083E007C09091DF05891302C084E001C002
:102C200081E00E94C7135092D302DF91CF911F9190
:102C30000F91FF90EF90DF90CF90BF90AF909F905B
:102C40008F907F906F905F900C94D301DF91CF9124
:102C50001F910F91FF90EF90DF90CF90BF90AF90BA
:102C60009F908F907F906F905F9008950E94AC141A
:102C70000E946406FBCFC8E0D4E088B38C2788BBF1
:102C80008091D702811102C0C29A08C088B38D27F3
:102C900088BB8091D70281508093D7028AEF90E061
:102CA0000E94F90DEACF26E030E061E070E080E0BC
:102CB00090E0E8B3AB01082E01C0440F0A94EAF794
:102CC0004E2748BB4FEF51EEE4E041505040E0400A
:102CD000E1F700C0000001968830910551F72150BE
:102CE000310929F70895EF92FF920F93F89483E941
:102CF00091E090931F0680931E0690932106809387
:102D00002006B89AB99ABA9ABB9ABC9ABD9ABE9A4A
:102D1000BF9A0E94A3140E9453160E94A3140E94FB
:102D2000651A0E94260484ED92E00E944D020E94E2
:102D30006D028093D20288EB91E09F938F9385E799
:102D400091E09F938F930E94011D9EE0E92E96E0F3
:102D5000F92E00E020E030E042E350E06CEE71E05C
:102D60008BE396E10E94C90A0E94751A0E94861A96
:102D700022E1E22E26E0F22E20E030E040EC50E0AE
:102D800063EF71E08EEF99E10E94C90A30E1E32E12
:102D900036E0F32E20E030E040EC50E067EF71E0E9
:102DA00086E396E10E94C90A0E943E010E947001DA
:102DB0000E94A20144E1E42E46E0F42E20E030E03F
:102DC00040E051E06EEF71E089E399E10E94C90AA9
:102DD0000F900F900F900F908091D202873481F462
:102DE0000E94101486E1E82E86E0F82E20E030E004
:102DF00040E053E062E072E08AE294E10E94C90A96
:102E00009EE088E10FB6F894A89581BD0FBE91BDF4
:102E100078940E94EE0B80E090E00F91FF90EF908D
:102E20000895C29885E691E09F938F930E94011DBB
:102E30000F900F900895C2987F936F938FE491E065
:102E40009F938F930E94011D80910E0690910F0613
:102E50000E9485101F928F938BE391E09F938F9335
:102E60000E94011D80911206909113060E94851008
:102E70001F928F938BE291E09F938F930E94011D8D
:102E800080911006909111060E9485101F928F93D9
:102E900089E191E09F938F930E94011D8091140618
:102EA000909115060E9485101F928F9389E091E002
:102EB0009F938F930E94011D8DB79EB744960FB6C6
:102EC000F8949EBF0FBE8DBF8091D202873491F4DB
:102ED00080911606909117060E9485101F928F937D
:102EE00088EF90E09F938F930E94011D0F900F90A9
:102EF0000F900F900895A8950895EF92FF920F9369
:102F00001F93CF93DF93EC01C59803EB14E0E12C02
:102F1000F12C48E050E0BE01C80142960E94F31C2B
:102F2000892B49F048E050E0BE01C8014B960E9451
:102F3000F31C892B29F4C7010E947E140E94D3013F
:102F400048E050E0BE01C8010E94F31C892B49F003
:102F500048E050E0BE01C80109960E94F31C892B8D
:102F600029F4C7010E946C140E94D3018FEFE81A64
:102F7000F80A0C5D1F4F88E0E816F10451F68091C5
:102F8000D202873409F055C048E050E0BE018AED16
:102F900092E00E94F31C892B11F40E940C0148E07E
:102FA00050E0BE0183EE92E00E94F31C892B21F4D5
:102FB00065E081E00E94B81348E050E0BE018CEE6D
:102FC00092E00E94F31C892B21F465E082E00E94CC
:102FD000B81348E050E0BE0185EF92E00E94F31C78
:102FE000892B11F40E940C0148E050E0BE018EEFE5
:102FF00092E00E94F31C892B21F465E084E00E949A
:10300000B81348E050E0BE0187E093E00E94F31C53
:10301000892B21F465E085E00E94B81348E050E078
:10302000BE0180E193E00E94F31C892B11F40E9401
:103030000C01C59ADF91CF911F910F91FF90EF90F6
:103040000895CF93DF93EC01C5988A819091D402C3
:10305000891305C02B819091D502291739F08E3242
:1030600009F07CC08B818E3209F078C08C81843469
:1030700089F130F48234B1F0F0F4813451F046C07B
:103080008634C1F170F1833E09F43FC0803FA9F15D
:103090003DC08D81803371F58E8190E0C0970E9494
:1030A0006C1415C08D81803329F58E8190E0C09716
:1030B0000E947E140CC08D818033E1F48E818033B8
:1030C00011F41BBA04C08133A9F48FEF8BBB0E94AB
:1030D000D3011CC08D81803369F48E81803351F41B
:1030E000F6CF8D81803331F48E8190E0C0970E94BD
:1030F0009114EDCF0E940C0109C08881833431F412
:10310000CE0105960E945E02FFCFFFCF8091D202D2
:10311000873421F5EC818E2F90E0FC01E156F10916
:10312000ED30F105D8F4E15BFF4F0C94B11A65E086
:1031300081E002C065E082E00E94B8130FC065E044
:1031400084E0FACF65E085E0F7CF0E940C0106C06D
:103150008FEF0E94D7018FEF0E941202C59ADF9174
:10316000CF910895AF92BF92CF92DF92EF92FF92EC
:103170000F931F93CF93DF93CDB7DEB72D970FB685
:10318000F894DEBF0FBECDBFFC01C598828190913F
:10319000D402891305C023819091D502291739F0F3
:1031A0008E3209F054C083818E3209F050C0848180
:1031B0008D3409F04CC08F018081833409F045C003
:1031C00040E150E060E070E0CF0107960E94D81B1C
:1031D0006B017C016115724081059105B0F5F80124
:1031E00095819E012F5F3F4F59019F3381F086816A
:1031F0008F3369F099838A831B8240E150E060E05D
:1032000070E0C9010E94D81BC6010E942404C601B7
:103210000E942204FF92EF92DF92CF921F928F932F
:1032200084ED92E09F938F938FE092E09F938F9332
:10323000BF92AF920E94271DC5010E946A190FB666
:10324000F894DEBF0FBECDBF02C00E940C01C59A2C
:103250002D960FB6F894DEBF0FBECDBFDF91CF9194
:103260001F910F91FF90EF90DF90CF90BF90AF90A4
:103270000895CF93DF93CDB7DEB72D970FB6F894AF
:10328000DEBF0FBECDBF8E010F5F1F4F8DE0F80177
:1032900011928A95E9F78DE0F82EC8010E948419F1
:1032A0008885843259F48981813521F4C8010E94CE
:1032B0007D170AC0C8010E94211806C08C8586327D
:1032C00019F4C8010E94B218F8018F2D11928A9545
:1032D000E9F7E3CFBC018091CE029091CF02009735
:1032E00029F020E04AE050E00C945F080895BC010A
:1032F0008091D0029091D102009729F020E040E027
:1033000050E00C945F080895BC018091D002909128
:10331000D102009721F04FEF5FEF0C94250908953B
:10332000C098C6985D9BFECF8CB9C09AC69A089586
:10333000CF93DF93EC018991882319F00E949019B3
:10334000FACFDF91CF910895C79890919B0095FF98
:10335000FCCF80939C00C79A0895CF93C82F8A30E2
:1033600019F48DE00E94A4198C2F0E94A41980E00A
:1033700090E0CF9108951F920F920FB60F921124F3
:103380008F93EF93FF93C098C698E091AD02EF5FE3
:10339000EF71E093AD028CB1F0E0E255FD4F808318
:1033A000C09AC69AFF91EF918F910F900FBE0F9028
:1033B0001F9018951F920F920FB60F9211248F93A2
:1033C000C79880919C00C79A8F910F900FBE0F9065
:1033D0001F901895E091AC02EF5FEF71E093AC02A3
:1033E000F0E0E255FD4F808108952091AD0290916B
:1033F000AC0281E0291301C080E00895CF93DF93F0
:10340000CDB7DEB76A970FB6F894DEBF0FBECDBF5B
:10341000E12CF12C00E010E0CE0101966C018DE072
:10342000B82E8091CE029091CF02009789F040E0B3
:1034300050E0BE01625F7F4F0E942509813041F458
:10344000CE010E960E94981985E090E00E94F90D39
:103450000E9464060E94F519882331F10E94EA193E
:10346000F601E00FF11F80830F5F1F4F843221F4BC
:103470000830110551F405C0863239F40C301105BD
:1034800021F4C6010E94771903C00D30110554F0D4
:10349000F6018B2D11928A95E9F7E12CF12C00E0D1
:1034A00010E002C0E12CF12C9FEFE91AF90AE1E0EB
:1034B000EE16FE0638F0F6018B2D11928A95E9F78B
:1034C00000E010E00E946406ACCF1092980083E008
:1034D00080939900EDE9F0E0808186608083EAE9DD
:1034E000F0E08081886980830895109290008CE0DC
:1034F00089B9E5E9F0E08081866080838AB18869D6
:103500008AB91092AC021092AD02089540E06DE0CD
:1035100080E10E9433089093D1028093D002892BDE
:1035200041F48CEB91E09F938F930E94011D0F90CB
:103530000F9040E06DE080E10E9433089093CF024D
:103540008093CE028091D0029091D102892B41F4D8
:103550008FE991E09F938F930E94011D0F900F9030
:103560000895EE0FFF1F0590F491E02D09940F933D
:103570001F93CF93DF938230910510F482E090E0A7
:10358000E0911A06F0911B0620E030E0A0E0B0E0E8
:10359000309719F1408151810281138148175907F1
:1035A000C8F08417950769F4109731F012960C93C0
:1035B000129713961C9327C000931A0610931B06AC
:1035C00022C02115310519F04217530718F49A014A
:1035D000BD01EF01DF01F801DBCF21153105F9F065
:1035E000281B390B2430310580F48A819B816115B9
:1035F000710521F0FB019383828304C090931B0625
:1036000080931A06FE01329644C0FE01E20FF31FBA
:103610008193919322503109398328833AC02091B4
:10362000180630911906232B41F4209102013091A4
:103630000301309319062093180620910001309160
:1036400001012115310541F42DB73EB74091040128
:1036500050910501241B350BE0911806F0911906D5
:10366000E217F307A0F42E1B3F0B2817390778F059
:10367000AC014E5F5F4F2417350748F04E0F5F1FB8
:1036800050931906409318068193919302C0E0E08D
:10369000F0E0CF01DF91CF911F910F910895CF936B
:1036A000DF93009709F481C0FC01329713821282E4
:1036B000A0911A06B0911B06109781F420813181E8
:1036C000820F931F20911806309119062817390789
:1036D00051F5F0931906E093180667C0ED0120E05C
:1036E00030E0CE17DF0740F44A815B819E0141152F
:1036F0005105F1F0EA01F5CFD383C28340815181B6
:10370000840F951FC817D90759F488819981840FB0
:10371000951F0296918380838A819B819383828304
:103720002115310529F4F0931B06E0931A063DC0DC
:10373000E901FB83EA8349915991C40FD51FEC1726
:10374000FD0761F480819181840F951F0296E90144
:1037500099838883828193819B838A83E0E0F0E070
:1037600012968D919C911397009719F0FD01DC0141
:10377000F7CF8D919C9111979D012E5F3F4F820F46
:10378000931F20911806309119062817390769F4FC
:10379000309729F410921B0610921A0602C0138269
:1037A0001282B0931906A0931806DF91CF91089565
:1037B000A0E0B0E0EEEDFBE10C946C205C016B014D
:1037C0007A016115710519F0FB0191838083E11481
:1037D000F10429F0C7010297839708F0C9C0E501F9
:1037E0002196F5011081812F90E00E94CD1C892B3C
:1037F00011F05E01F4CF1D3229F42196F5011181FB
:1038000001E007C01B3221F4E5012296F501118188
:1038100000E0E114F104B1F0F0E1EF16F10429F455
:10382000B0C010E3E114F10401F12AE0E216F10462
:10383000B1F180E1E816F10471F0E8E0EE16F10470
:10384000F1F413C0103341F588818F7D883549F735
:10385000198122960260F0E1EF2EF12C88248A94DF
:10386000982CA82CAFE0BA2E20C078E0E72EF12CDF
:1038700088248A94982CA82CEFE1BE2E16C06FEFF6
:103880007FEFCB0197010F2C000C440B550B0E94CE
:103890003E2049015A0109C08AE0E82EF12C69E96D
:1038A000862E982CA82C69E1B62E40E060E070E0EE
:1038B000CB0127010F2C000C66087708FE0150EDA4
:1038C000352E310E29E0231570F42FEB210F2A310C
:1038D00018F439EC332E06C02FE9210F2A3130F5C8
:1038E00029EA322E310E232D30E02E153F05F4F457
:1038F0004F3FC9F086169706A806B90688F0A301BF
:1039000092010E942E20232D30E040E050E0620F13
:10391000731F841F951F621773078407950710F4A0
:103920004FEF01C041E021961081C8CFC114D104EE
:1039300051F0442311F0219703C001FF04C02297E6
:10394000F601D183C08300FF07C0909580957095E4
:1039500061957F4F8F4F9F4F4F3F79F482E290E008
:1039600090932306809322063FEF2FEF9FEF0DC029
:1039700040E030E020E090E008C0462F372F282FAD
:1039800004C0103309F067CF5FCF642F732F822FED
:10399000CDB7DEB7E1E10C94882091110C944C1F57
:1039A000803219F089508550C8F70895FB01DC0179
:1039B00004C08D910190801921F441505040C8F706
:1039C000881B990B0895FB01DC0102C001900D9248
:1039D00041505040D8F70895DC0101C06D9341502B
:1039E0005040E0F70895FB01DC014150504030F0B9
:1039F0008D910190801919F40020B9F7881B990B5B
:103A00000895A0E0B0E0E7E0FDE10C947920AE017C
:103A1000495F5F4FDA016D917D91AD010CE116E0D8
:103A2000F80182819381DC0113962C911397286011
:103A300013962C930E946B1DD8011296ED91FC9168
:103A400013972381277F2383E4E00C949520AEE035
:103A5000B0E0EDE2FDE10C9479200D891E8986E04D
:103A60008C831A8309838FEF9FE79E838D83AE013A
:103A7000475E5F4F6F89788DCE0101960E946B1D66
:103A8000EF81F885E00FF11F10822E96E4E00C9490
:103A90009520AEE0B0E0EFE4FDE10C9479200D89D3
:103AA0001E898EE08C831A8309838FEF9FE79E83A4
:103AB0008D83AE01475E5F4F6F89788DCE01019691
:103AC0000E946B1DEF81F885E00FF11F10822E968A
:103AD000E4E00C949520ABE0B0E0E1E7FDE10C946C
:103AE0006B206C017B018A01FC01178216828381A5
:103AF00081FFCCC1CE0101963C01F6019381F70113
:103B000093FD859193FF81917F01882309F4BAC1C8
:103B1000853239F493FD859193FF81917F01853240
:103B200029F4B60190E00E94651FE7CF912C212C6B
:103B3000312CFFE1F315D8F08B3279F038F4803274
:103B400079F08332A1F4232D20611DC08D3261F004
:103B5000803369F4232D216016C0832D8260382EB6
:103B6000E32DE4603E2E2AC0F32DF8601DC037FC23
:103B70002DC020ED280F2A3040F08E32B9F436FCEB
:103B800081C1232D2064322E19C036FE06C08AE082
:103B9000989E200D1124922E11C0EAE02E9E200D39
:103BA0001124222EF32DF0623F2E08C08C3621F412
:103BB000832D8068382E02C0883641F4F70193FDCA
:103BC000859193FF81917F018111B3CF982F9F7DC4
:103BD0009554933028F40C5F1F4F9FE399830DC0D9
:103BE000833631F0833771F0833509F059C021C035
:103BF000F801808189830E5F1F4F88248394912C64
:103C0000530113C02801F2E04F0E511CF801A080AF
:103C1000B18036FE03C0692D70E002C06FEF7FEF08
:103C2000C5010E945A1F4C018201F32DFF773F2EE0
:103C300016C0280122E0420E511CF801A080B1807C
:103C400036FE03C0692D70E002C06FEF7FEFC50143
:103C50000E944F1F4C01F32DF0683F2E820133FC70
:103C60001BC0822D90E088169906B0F4B60180E260
:103C700090E00E94651F2A94F4CFF50137FC8591EE
:103C800037FE81915F01B60190E00E94651F21100F
:103C90002A9421E0821A91088114910471F7E8C0F6
:103CA000843611F0893641F5F80137FE07C060818E
:103CB0007181828193810C5F1F4F08C06081718187
:103CC000072E000C880B990B0E5F1F4FF32DFF760C
:103CD0003F2E97FF09C090958095709561957F4F15
:103CE0008F4F9F4FF0683F2E2AE030E0A3010E94E3
:103CF000A11F882E861845C0853731F4232D2F7ECD
:103D0000B22E2AE030E025C0932D997FB92E8F3650
:103D1000C1F018F4883579F0B5C0803719F08837CC
:103D200021F0B0C0E92FE061BE2EB4FE0DC0FB2D26
:103D3000F460BF2E09C034FE0AC0292F2660B22EBF
:103D400006C028E030E005C020E130E002C020E1FC
:103D500032E0F801B7FE07C06081718182819381F2
:103D60000C5F1F4F06C06081718180E090E00E5FA4
:103D70001F4FA3010E94A11F882E8618FB2DFF77DD
:103D80003F2E36FE0DC0232D2E7FA22E891458F40F
:103D900034FE0BC032FC09C0832D8E7EA82E05C0D8
:103DA000B82CA32C03C0B82C01C0B92CA4FE0FC0A2
:103DB000FE01E80DF11D8081803321F49A2D997E5A
:103DC000A92E09C0A2FE06C0B394B39404C08A2DE4
:103DD000867809F0B394A3FC11C0A0FE06C0B2140B
:103DE00088F4280C922C9B180EC0B21460F4B60113
:103DF00080E290E00E94651FB394F7CFB21418F4EC
:103E00002B1802C0982C212CA4FE10C0B60180E310
:103E100090E00E94651FA2FE17C0A1FC03C088E7C6
:103E200090E002C088E590E0B6010CC08A2D86784B
:103E300059F0A1FE02C08BE201C080E2A7FC8DE236
:103E4000B60190E00E94651F891438F4B60180E342
:103E500090E00E94651F9A94F7CF8A94F301E80DD1
:103E6000F11D8081B60190E00E94651F8110F5CFA1
:103E7000222009F442CEB60180E290E00E94651F44
:103E80002A94F6CFF6018681978102C08FEF9FEFCB
:103E90002B96E2E10C948720992788270895FC014E
:103EA0000590615070400110D8F7809590958E0F65
:103EB0009F1F0895FC016150704001900110D8F7D8
:103EC000809590958E0F9F1F08950F931F93CF930A
:103ED000DF93FB01238121FD03C08FEF9FEF2CC0F7
:103EE00022FF16C04681578124813581421753072E
:103EF00044F4A081B1819D012F5F3F4F3183208326
:103F00008C93268137812F5F3F4F3783268314C0E0
:103F10008B01EC01FB010084F185E02D0995892BD3
:103F2000E1F6D80116968D919C91179701961796F8
:103F30009C938E931697CE01DF91CF911F910F9195
:103F40000895FA01AA27283051F1203181F1E8942F
:103F50006F936E7F6E5F7F4F8F4F9F4FAF4FB1E07C
:103F60003ED0B4E03CD0670F781F891F9A1FA11D77
:103F7000680F791F8A1F911DA11D6A0F711D811D78
:103F8000911DA11D20D009F468943F912AE0269F3D
:103F900011243019305D3193DEF6CF010895462F9C
:103FA0004770405D4193B3E00FD0C9F7F6CF462F7D
:103FB0004F70405D4A3318F0495D31FD40524193E6
:103FC00002D0A9F7EACFB4E0A695979587957795A3
:103FD0006795BA95C9F700976105710508959B012A
:103FE000AC010A2E06945795479537952795BA95B3
:103FF000C9F7620F731F841F951FA01D0895DC0170
:10400000CB01FC01E199FECF06C0FFBBEEBBE09AFD
:1040100031960DB20D9241505040B8F70895E19994
:10402000FECF9FBB8EBBE09A99278DB30895DC012C
:10403000CB0103C02D910E94222041505040D0F767
:104040000895262FE199FECF9FBB8EBB2DBB0FB6E7
:10405000F894E29AE19A0FBE01960895DB018F93DE
:104060009F930E946020BF91AF91A29F800D911DF0
:10407000A39F900DB29F900D11240895A1E21A2ED6
:10408000AA1BBB1BFD010DC0AA1FBB1FEE1FFF1FFC
:10409000A217B307E407F50720F0A21BB30BE40B4C
:1040A000F50B661F771F881F991F1A9469F7609593
:1040B0007095809590959B01AC01BD01CF0108954D
:1040C0000E94A220A59F900DB49F900DA49F800DEB
:1040D000911D112408952F923F924F925F926F92FB
:1040E0007F928F929F92AF92BF92CF92DF92EF9288
:1040F000FF920F931F93CF93DF93CDB7DEB7CA1B09
:10410000DB0B0FB6F894DEBF0FBECDBF09942A8833
:10411000398848885F846E847D848C849B84AA84DB
:10412000B984C884DF80EE80FD800C811B81AA8168
:10413000B981CE0FD11D0FB6F894DEBF0FBECDBF33
:10414000ED010895A29FB001B39FC001A39F700D20
:10415000811D1124911DB29F700D811D1124911D8F
:064160000895F894FFCF62
:10416600000024062000040205006113D6050203A0
:10417600006113D6050201006113D705020201771B
:1041860013D4050204006113D7050105009113D667
:10419600050103013A1300000101009113D705013F
:1041A60002009113D6050104009113D705040501F9
:1041B6003C1300000403013C1300000401013C13FE
:1041C60000000402013C1300000404013C1300003B
:1041D6000505006113D6050503006113D605050123
:1041E600006113D7050502017713D50505040061A3
:1041F60013D7050000000200000000AD1900000002
:1042060000513F2E2E3F3F3F24000058582E2E3F90
:104216003F3F2400002A2A005330343038473334D5
:104226000049444C4500092563092575092575098A
:1042360025750D0A00546D725100546D7220537627
:1042460063006761746554696D65720072756E4CC2
:1042560045440052434D00496E70757473005543D2
:10426600530047617465002573202564200A0025E4
:10427600732E2E50253032582530346C58260000C7
:00000001FF
